:1021D8005553422D44494F2D3332005553422D4417
:1021E800494F2D3234005553422D4F544845520023
:10167000EF75F00CA4248CF582E43428F58375F022
:1016800004EE120517E4F0EEC4333354C04432FDC7
:10169000EF75F00CA4248BF582E43428F58375F003
:1016A00004EE020517F0A374FFF0A3F0A3F0A3F07B
:1016B00022E0F580A3E0F590A3E0F5A0A3E0F5B06B
:1016C00022E490E68AF090E6BEE090E68BF022AB52
:0816D0002AAA2BA92C02043AFE
:04002E0043B1202298
:0400460053B1DF22B1
:04004E0063B1202258
:0100320022AB
:101C57007AE779407F40AB077D017F037E00121D45
:101C67008090E740E0FF90010CF024FB600C240417
:101C770070107BFF7A2179D8800E7BFF7A2179E378
:0C1C870080067BFF7A2179EE12190A22F8
:10209E00902806E0600312173B902808E0600312B8
:1020AE001AA390281AE06003121B8790285CE06048
:0B20BE000990281BE06003121961224A
:03004000021C5748
:01004A002293
:01005200228B
:012464002255
:10185800EF5407FE7401A806088002C333D8FCFEC3
:10186800EF131313541FFFED601EEF14600E146086
:101878000F14601024037031EE428022EE42902251
:10188800EE42A022EE42B022EF14600F1460111451
:10189800601324037013EEF4528022EEF452902267
:0A18A800EEF452A022EEF452B0223A
:101C9300EF54F824F8601024F8601024F86010243E
:101CA30018700EAE80800AAE908006AEA08002AEA1
:101CB300B0EF5407FF7401A807088002C333D8FCB0
:0C1CC3005206EE60047F0180027F0022C8
:10000E00E580120480900001E590120492900002A7
:0D001E00E5A0120492900003E5B0020492E8
:101FEB0012043A90285EF0F5809000011204539091
:101FFB00285FF0F590900002120453902860F0F5E2
:0E200B00A0900003120453902861F0F5B0225B
:1018B2008B2A8A2B892C12043AFF30E0047EFF80A7
:1018C200027E008EB2EF30E1047FFF80027F008F44
:1018D200B31216CFFF30E2047EFF80027E008EB488
:1018E200EF30E3047FFF80027F008FB5AB2DAA2E7D
:1018F200A92F12043A5401C454F0FF1216CF540F08
:081902004F90285DF0F5B122C1
:10157F007E007FAF7D007B017A287900120576907F
:10158F002800740AF0E41216AA90285D1216A5E43A
:10159F009028861216A5E4902805F0902804F09064
:1015AF002807F0902806F0902808F0A3F090281A4A
:1015BF00F0A3F090285CF0FFE4FEEF75F00CA4248C
:1015CF0063F582E4342812169CE4F0EEC4333354EE
:1015DF00C04432FDEF75F00CA42462F582E4342888
:1015EF0012169CEDF0121670EDF00EBE03CC0FEF3D
:0515FF00640370C4222A
:101A050090E600E054E7F075B63F90285E1216B1F7
:101A150090285DE0FF30E0047EFF80027E008EB2FC
:101A2500EF30E1047FFF80027F008FB390285DE0F7
:101A3500FF30E2047EFF80027E008EB4EF30E304C7
:101A45007FFF80027F008FB590285DE0F5B102240D
:011A5500147C
:1023D1008F248D253006030201E2AD25AF241202C0
:0223E1000122D7
:012465002254
:012466002253
:10234F009028861216A7E4FFE4FE121670EDF00E29
:08235F00BE02F70FBF03F122DB
:101A56009028871216B1902886E0FF30E0047EFFBA
:101A660080027E008EB2EF30E1047FFF80027F00AD
:101A76008FB3902886E0FF30E2047EFF80027E006E
:101A86008EB4EF30E3047FFF80027F008FB590288D
:0D1A960086E0F5B17B017A28798B021604F9
:1011BD00D204120B0C500302127490E6B9E024ED28
:1011CD00600E24E3607214606F241F6003021272BC
:1011DD0090E6B8E030E723E5B1540F90E740F0E535
:1011ED00B130E4047F0180027F0090E741EFF07B96
:1011FD00017AE7794212000E805F1216C190E6A0C7
:10120D00E020E1F990E6BDE0FF90E6BCE04F700B09
:10121D00752D01752EE6752FBA8009752D01752E68
:10122D00E7752F417B017AE779441218B27B017A79
:10123D00E77940121FEB802F7B017AE7794012008E
:10124D000EE5B1540F90E744F0E5B130E4047F01B1
:10125D0080027F0090E745EFF01216C190E6A0E006
:09126D004480F08002D322C32268
:1001020012010002000000400516018001000102F8
:020112000001EA
:0A0116000A0600020000004001008C
:1001220009022000010100A0FA0904000002FF00F8
:100132000000070502020002000705860200020015
:1001440009022000010100A0FA0904000002FF00D6
:10015400000007050102400000070581024000007D
:100166001403000000000000000000000000000072
:1001760000000000260341004300430045005300F1
:10018600200049002F004F002000500072006F0031
:10019600640075006300740073002003550053006B
:1001A60042002D00440049004F002D00330032006C
:1001B6000000000000000000000000008081828333
:1001C600848586879091929394959697A0A1A2A3F1
:1001D600A4A5A6A7B0B1B2B3B4B5B6B7C0D0C0E0B7
:1001E600EF9001C2939001F9F0ED9001C293900156
:1001F600FBF0A2009200D0E0D0D022C0D0C0E0EF49
:100206009001C293900218F0ED9001C29390021BE8
:0B021600F0A200B39200D0E0D0D02294
:10231B00564A616E20323520323031384031333AF3
:0B232B0035383A333800000000000095
:102394000217233202080000010F01010C01010A97
:0423A400010114FF20
:1008F900E0FFAE2F052F74402EF582E434E7F5832F
:100909002275F00CE542120517E54175F00CA42596
:1009190083F583E5822FF582E5833EF58322E49012
:10092900E68AF090E6BEE090E68BF022EC75F008DE
:10093900A4FFED7A002FFFEA35F0FEE42FF582746B
:10094900803EF5832275F009E52BA4F58285F083B5
:1009590075F003E52D120517E5822290E740F0E4D2
:1009690090E68AF090E68B22E0FE74D32FF582E4BC
:100979003428F583E022FF7444252BF582E434E71B
:10098900F583EFF0052BE52B22AA39A93A75F00C6E
:10099900E53CA4F58285F08375F004E53B12051763
:1009A900020453FF7E000DEE2518F582E43517F594
:1009B900832275F008A42403F582E5F03480F583D9
:1009C90022252FF52FE532352EF52EC3E531953346
:1009D900F531E5309532F5302274402535F58274CC
:1009E900E73534F583227586005391EF90E65D2251
:1009F90024867C007B01F9EC22E490E68BF090E6FA
:100A0900BAE0FFA3E02235F0FAE53B75F004A4292A
:100A1900F9EA35F0FA2274DD252BF582E43428F55C
:100A29008322EC25E0240AF582E43428F583E0FEEC
:100A3900547FFFEE2274B32FF582E43428F5832224
:100A490074AF2EF582E43428F583E0227DAF7A284D
:100A59007B007F017E1F22E4F512F513F519F51AC3
:100A69002290E6BEE0640122C3E5359533E534956D
:100A7900322274D92FF582E43428F5832290E6BE18
:100A8900E0640222F583EFF090E741E0FFEE25E014
:100A990022E52F2535F582E52E3534F58322854C5F
:100AA90050854D518554528555532285545085554D
:100AB90051854C52854D5322AC07C413135403FD81
:100AC90022AF047E007C00754700F5482290E6A01D
:100AD900E04480F02275F00CE53E120517E53D2251
:100AE900AD337AE77B40AF2FAE2E22902800740AEF
:100AF900F0E4A3F0227C007B01F9EC227B017AE788
:030B09007940220E
:1020C9008B3FA905E9120AC1EC1209BBE9F0120913
:1020D90035E53FF0120944E540F0AB01E53F120A4E
:0B20E900CAE540754900F54A021C18CA
:10237F00AB05EB120AC3EF1209BBEBF07E007C003A
:05238F007A0002201994
:10216D008D2FA903E52F120AC1120935E9F01209C5
:10217D0044E531F0AB2FE9120ACAE531754900F596
:04218D004A021C18CE
:1016D800A9077401A805088002C333D8FC25E04493
:1016E800C0FF75F008E91209BEEFF0E975F008A42B
:1016F800FFED7583002FFFE583120941E0FC74427A
:101708002BF582E434E7F583ECF0120944E0FF742A
:10171800402B120902EFF0E975F008A47C002DFFB8
:10172800EC120941E0FF74412BF582E434E7F583BC
:03173800EFF022AD
:101604008B388A39893AE4F53CE4F53BE53C75F0DE
:101614000CA4AB38253AF9E539120A0F90000112EF
:101624000453602A120992FCE53C75F00CA429F9D4
:10163400EA120A0F900002120453FD9000031204F0
:1016440053F540AB05AD04AF3C1220C9800BAB3859
:10165400120992FDAF3C12237F053BE53BC3940284
:0C16640040AA053CE53CC39403409E22D4
:10233600902803E0FF7006902802E06008902802CB
:09234600E0FD0200E4122457221C
:1022CA007E007FAF7D007B017A28790012057612A5
:0B22DA000AF412157F121A050223E31C
:1021F8007D02120A57121D80902800E0B40A04A339
:10220800E060030222CA120A55121D80121A052222
:1023E300120AF4120A55121E5D7DAF7F007E1F0292
:0223F300245470
:10179E0012233690E6BEE0F539753B02E539604B13
:1017AE00C39440500585393A8003753A4012096852
:1017BE00E53AF090E6A0E020E1F9E4F538E538C32B
:1017CE00953A501E74402538120902E0FFAE3B05D3
:1017DE003BEE24001209FB3428FAEF120480053880
:0E17EE0080DBC3E539953AF53980B102233628
:092414007B017A287962021604AA
:101C18008E418F428C438D448A458B46E544AE43C2
:101C28007802C333CE33CED8F9FF90286312090A5D
:101C38007401F090286412090AE548F090286512AA
:0F1C4800090AE54AF090286212090AE546F022DF
:102019008E3D8F3E8C3F8D40E540AE3F7802C33305
:10202900CE33CED8F9FF902863120ADE120914E4E0
:0D203900F0902862120ADE120914EBF0226A
:1012760090E6B8E030E733E4F52FF52EE52EC3947B
:101286002950207E007B01745D252EF9EE3428FA64
:1012960012043AFF7440252F120902EFF0052E05BD
:1012A6002F80D9120927120AD62212092C90E6A0FD
:1012B600E020E1F990E6BEE064296003C20422E47E
:1012C600F52EF52FE52EC39429501D7440252F12B7
:1012D6000902E0FFE52E245D120AFE3428FAEF1219
:1012E6000480052E052F80DC90E6BAE0B4CE08A374
:0812F600E0B4AC031223E32273
:0F240500D3E51A950EE519950D400312241D22FB
:012467002252
:1021B500902805E0FE902804E07C002400F50EEC54
:1021C5003EF50D450E7007C28CC2A9C20522D28C00
:0321D500D2A9226A
:012468002251
:101D460012092C90E6A0E020E1F9E4FF74422FF599
:101D560082E434E7F583E0FEEF1209F93428FAEE5F
:101D66001204800FBF29E590E740E0902804F09028
:0A1D7600E741E0902805F00221B5D6
:09241D00121A56120A60D20522BF
:10236700C205120A60C28CC2A9538EF75389F14382
:0823770089011224680221B55E
:101DF100E50945086019E50915097002150814C3BC
:101E010094FFE508648094805016120046801130DA
:101E1100040E7508057509FF12002EC204120A602E
:061E2100300502D204228C
:1010EA0090E6B8E030E75CE4F52F9028041208F99E
:1010FA00EFF09028051208F9EFF0E4F52EE52EC37B
:10110A00942950207E007B017486252EF9EE34281E
:10111A00FA12043AFF7440252F120902EFF0052E45
:10112A00052F80D91208FBE51AF0E5191208FAEF23
:10113A00F0A205E4331208FAEFF0C20512092712E9
:10114A000AD62212092C90E6A0E020E1F9C2059005
:10115A00E6BEE0642B6003C20422E4F52FAF2F053C
:10116A002F74402F120902E0902804F0AF2F052FA8
:10117A0074402F120902E0902805F0E4F52EE52EBE
:10118A00C39429501B7440252F120902E0FFE52E53
:10119A001209F93428FAEF120480052E052F80DE91
:1011AA001221B590E6BAE0B4CE08A3E0B4AC0312BB
:0311BA0023E3220A
:04244800750F0122E9
:1017FC0012233690E6BEE0F539E4F53BE539604B53
:10180C00C39440500585393A8003753A40120968F3
:10181C00E53AF090E6A0E020E1F9E4F538E538C3CC
:10182C00953A501E74402538120902E0FFAE3B0574
:10183C003BEE241B120AFE3428FAEF120480053802
:0C184C0080DBC3E539953AF53980B12204
:10196100150FE50F704B90281BE0F50F122465E46D
:10197100F52190285CE0FFE521C39F5031E5212549
:10198100E0241CF582E43428F583E0F522E52125E5
:10199100E0241DF582E43428F583E0F523547FFD2E
:1019A100E523339206AF221223D1052180C41224EC
:0219B1006622AC
:1022E50012092C90E6A0E020E1F990E740E0902863
:0B22F50006F090E741E0902807F0227F
:10173B00150CE50C705C902806E0F50C7B017A2803
:10174B0079E112000EE4FFFE74E12EF582E43428F9
:10175B00F583E0FD120A496DF97D01E4FCECC394BD
:10176B00085029E95D6013120A3EE014F0120A3E9C
:10177B00E07011120A496DF08000902807E0FB120F
:10178B000A3EEBF00CED25E0FD0F80D10EEE64046C
:03179B0070B62203
:1023BE0012092C90E6A0E020E1F990E740E0902889
:0323CE0008F022F2
:10225600E4F515FF120973FE74DD2F120A23EEF062
:0E226600120973FE120A7BEEF00FBF04E7228E
:101AA300150AE50A7045902808E0F50A7B017A28B3
:101AB30079D312000EE4FF74DD2F120A23C083C012
:101AC30082120971FDEE5DD082D083F0120A7BC0D1
:101AD30083C082120971FDEE4DD082D083F00FBF17
:0C1AE30004D5E515C394FF500205152240
:04244C007514FF22E2
:101B8700E4FC051490281AE0FFECC39F5032EC25C3
:101B9700E0240BF582E43428F583E0C39514500E56
:101BA700120A2B30E7047D0080107D01800C120A99
:101BB7002B30E7047D0180027D001218580C80C489
:0B1BC700902809E0B51403E4F5142297
:10211F0012092C90E6A0E020E1F9E4FF74402F12A1
:10212F000902E0FEEF7C007B012409F9EC3428FA68
:09213F00EE1204800FBF12E4222D
:100056008E388F39E4F53AE53964024538700C90EC
:10006600E741F0E539153970021538E5396401457F
:1000760038701090E74074AF12092BE539153970C6
:10008600021538E5394538605490E6A0E020E1F9DC
:10009600C3E5399440E53894005004AD3980027DBB
:1000A60040E4FFEFC39D5021AE3A053AEE7583005A
:1000B6007B012400F9E5833428FA12043AFE7440E1
:1000C6002F120902EEF00F80DA120968EDF0FFC375
:0E00D600E5399FF539E5389400F53880A6220B
:1005A20090E6B8E030E76090E6BFE0FE90E6BEE09D
:1005B200FDEDFF4E7002804A90E6BDE0FD90E6BC84
:1005C200E04D700302005690E6BDE060030208F8B9
:1005D20090E6BCE01460030208F8753BFF753C230B
:1005E200753D1B753E00753F1E7B017AE77941120E
:1005F20019B3120B051223A9EF0490E740F090E61D
:10060200BEE090E68BF02290E6BFE0FF90E6BEE00F
:100612004F707790E6BDE0704D90E6BCE024EF604D
:1006220023249F603024FD603324F36034247270ED
:100632003590E6BAE064CE702DA3E064AC70271268
:1006420023E3802290E6BAE0B4CE1BA3E0B4AC165A
:100652001222CA8011E490281AF0800A7514FF80D1
:1006620005E490285CF090E6BDE064806003020837
:10067200F890E6BCE0640160030208F890E6BAE094
:10068200902802F090E6BB02074B90E6BFE06003C1
:100692000208F890E6BDE0FE90E6BCE07C00240093
:1006A200FFEC3EFEEF8EF012054906F4002006F440
:1006B200002106F4002206F400230729002F075325
:1006C200004107610051076C0053078900610794DC
:1006D200006307B1007107BF007307DC00740821D3
:1006E2000081082F0083084C0084089280010000DA
:1006F20008F890E6BEE0B4AD0312179E90E6BCE0A7
:1007020030E003121A0590E6BCE020E1030208F88B
:1007120090E6BAE064CE60030208F8A3E064AC603D
:10072200030208F80223E3120A8660030208F8E0D3
:1007320090E68BF090E6A0E020E1F912233690E7F4
:1007420040E0902802F090E741E0902803F0020890
:10075200F590E6BEE0642B60030208F8021D461223
:100762000A8660030208F80222E5120A6A6003029E
:1007720008F8E090E68BF090E6A0E020E1F990E73F
:1007820040E0902806F022120A6A60030208F8028A
:1007920023BE120A6A60030208F8E090E68BF0902A
:1007A200E6A0E020E1F990E740E0902808F02290EE
:1007B200E6BEE0641260030208F802211F120A6A10
:1007C20060030208F8E090E68BF090E6A0E020E1FA
:1007D200F990E740E0902809F022120A86600302AD
:1007E20008F890281AE0C3940840030208F8120996
:1007F2002C90E6A0E020E1F990E740E0FF90281A73
:10080200E0FE25E02408F582E43428120A8D24094A
:10081200F582E43428F583EFF090281A02088E90CE
:10082200E6BEE0644260030208F80217FC120A6A9C
:1008320060030208F8E090E68BF090E6A0E020E189
:10084200F990E740E090281BF022120A866003022A
:1008520008F890285CE0C3942040030208F81209CB
:100862002C90E6A0E020E1F990E740E0FF90285CC0
:10087200E0FE25E0241AF582E43428120A8D241BB6
:10088200F582E43428F583EFF090285CE004F0224E
:1008920012092C90E6A0E020E1F990E6BEE06404A3
:1008A200705490E740E0FCA3E0FDA3E0FEA3E0F576
:1008B200318E308D2F8C2EFBAA30A92FA82E7F00CF
:1008C2007E1B7D377C4B12031C8F358E348D338C0F
:1008D20032AB35AA34A933A832E4FFFE7D807C47CF
:1008E2001202241203B98E368F37EF902802F0E5F8
:0708F20036A3F012233622A9
:1023000090E6047480F00000007402F00000007495
:0B23100006F0000000E4F000000022D6
:012469002250
:101D0B00E4F52A7AE779407F40AB077D087FF87EC0
:101D1B001D121D80E4F52A7440252A120902E0FDEC
:101D2B00E52A75F002A42468F9740135F08982F56F
:0B1D3B0083EDF0052AE52AB408DD2244
:101CCF0090E678E05410FFC4540F4450F51013E41D
:101CDF0033F516438E20120032122440121D0B12C0
:101CEF000040D2001221F812236712244812225604
:0C1CFF0012244C12233612004602004A48
:10227400120052121DF1122405E5B190E68020E708
:0E22840006E04408F08004E054F7F002246401
:10190A008B2A8A2B892CE4F52D1223A98F2EE52EFA
:10191A0025E024029001A0F0E4F52DAF2EEF3395D7
:10192A00E0FEC3E52D9FEE6480F87480985027ABE3
:10193A002AAA2BA92C852D82758300120453FDE552
:10194A002D75F002A424A2F9740135F08982F58379
:07195A00EDF0052D80C52210
:101DB9008E3E8F3FAC05E4FDE5166007E53E12094E
:101DC900ACEFF0AE050DE5182E1209B3E53FF0AF03
:101DD900050DE5182F1209B3ECF0AB18AA17AF10CF
:081DE9001222AEAF10021E270A
:03245400021DB9AD
:101E5D008E388F398D3A8A3B8B3CE4F53DE53DC399
:101E6D00953A50200539E539AE387002053814FF22
:101E7D00E53C253DF582E4353BF583E0FD12245428
:051E8D00053D80D92293
:101D80008E368F378D388A398B3AE4FDF53BE51670
:101D90006007E5361209ACEFF0AE050DE5182E121E
:101DA00009B3E537F0AB18AA17AF101222AEAB3A61
:091DB000AA39AD38AF10022292ED
:100EC60090E6BAE0752E00F52FA3E0FEEE422E90D6
:100ED600E6BEE0753000F531A3E0FEEE423090E666
:100EE600B8E064C06003020F8CE531453070030240
:100EF6000FE190E6A0E020E1F9C3E5319440E5304A
:100F0600940050088530328531338006753200757D
:100F1600334090E6B9E064A3704090E6BCE0B401CB
:100F26001BA3E0701790E6BBE030E71090E7407433
:100F360003F0A37401F0A37403F0803EE4F534F5E6
:100F460035120A715034120A9AE0FF1209E2EFF0E4
:100F56000535E53570EB053480E7E4F534F53512F3
:100F66000A7150101209E274CDF00535E53570EFBF
:100F7600053480EB120AE9121D80120968E533F088
:100F86001209CA020EEF90E6B8E06440704DE531F2
:100F960045306047120968F090E6A0E020E1F9903C
:100FA600E68BE0753200F53390E6B9E0B4A31EE4B3
:100FB600F534F535120A71501A1209E2E0FF120AE9
:100FC6009AEFF00535E53570EB053480E7120AE94E
:0C0FD600121E5DE5331209CA020F9422BE
:0212FE00C32209
:02245A00D3228B
:02245C00D32289
:0800030090E6BAE0F50BD322F0
:09242600E50B12096404F0D32255
:0824380090E6BAE0F511D32291
:09242F00E51112096404F0D32246
:02245E00D32287
:02246000D32285
:02246200D32283
:1013B800E4FF90E6B8E020E7030214640F0F7440DE
:1013C8002401120902740AF00F744024021209025F
:1013D800E4F00F74402403120902E4F00F7440246F
:1013E800041209027401F00F7440240512090274F2
:1013F80004F00F744024061209027403F00F7440BD
:101408002407120902E4F00F744024081209027438
:10141800FFF00F7440240912090274FFF00F7440A2
:10142800240A1209027408F00F7440240B120902EE
:101438007420F00F7440240C120902741FF00F740A
:1014480040240D120902741FF00F7440240E120973
:0D145800027401F090E740EFF01209272226
:100B0C0090E6B9E01205230B65100B65110B9E14D2
:100B1C000C0F150C6D200C7F210C89220CA0230CC2
:100B2C002E250CA0270B53280B4D2E0B473C0B5F8F
:100B3C003F0B59A20B59A300000D181205A2020D70
:100B4C001A1210EA020D1A121276020D1A120EC6A1
:100B5C00020D1A1213B8020D1A90E6B8E030E7092C
:100B6C00120B0512000E020C2790E6BEE0701090DE
:100B7C00E6BCE0FF90E6BAE0FD121858020D1A121E
:100B8C00092C90E6A0E020E1F9120B05121FEB02F4
:100B9C000D1AC2AF90E750E515F0E4F5157B017A1C
:100BAC00E7794C12000EE4F52B74D3252B12097641
:100BBC00FF7440252B12090212098BB404EB90E64A
:100BCC00BCE06010E4F52B120A1FE0F412097FB4AC
:100BDC0004F5800DE4F52B120A1FE012097FB40412
:100BEC00F6E4F52B74D9252B120A7EE0FF74482508
:100BFC002BF582E434E7120989B404E8122256D2A8
:100C0C00AF8018E4F52B74AF252B120A4CFF7440FF
:100C1C00252B12090212098BB404EBE490E68AF03E
:100C2C00804890E6BEE0B41B047F0180027F008FF9
:100C3C002AE4FAF52CE4F52BE52BC39403501CAFF6
:100C4C0002AB2CAD2B1216D8052BE52A60047F03C2
:100C5C0080027F02EF252CF52C80DD0ABA03D680AA
:100C6C0009120A07FDE4FB1216D812092C120AD637
:100C7C00020D1A120A02FD12237F020D1A120A0229
:100C8C00FEC413135403FDA3E0FBA3E0F5311221C2
:100C9C006D020D1A90E6BEE07011120A07FDA3E07A
:100CAC00FBA3E0F5401220C9020D1A90E6BEE064E9
:100CBC001B705BE090E68BF090E6A0E020E1F9E49D
:100CCC00F52BE4F52D12094E2440F582E58334E72B
:100CDC00F583E0FD12094E2441F582E58334E7F5F6
:100CEC0083E0FB12094E2442F582E58334E7F58359
:100CFC00E0F540AF2B1220C9052DE52DC394034020
:100D0C00C4052BE52BC3940340B88002C322D32225
:1020F400C0E0C083C082C085C084C086758600905D
:10210400E6B5E04401F0D2011209F27401F0D08680
:0B211400D084D085D082D083D0E03290
:10221800C0E0C083C082C085C084C0861209EF7444
:0F22280004F0D086D084D085D082D083D0E0322D
:10223700C0E0C083C082C085C084C0861209EF7425
:0F22470002F0D086D084D085D082D083D0E03210
:101EF800C0E0C083C082C085C084C086758600905B
:101F0800E680E030E705120AA78003120AB4120936
:101F1800F27410F0D086D084D085D082D083D0E0FF
:011F28003286
:10219100C0E0C083C082C085C084C086758600D27D
:1021A100031209F27408F0D086D084D085D082D091
:0421B10083D0E032C5
:101F2900C0E0C083C082C085C084C0867586009029
:101F3900E680E030E705120AA78003120AB4120905
:101F4900F27420F0D086D084D085D082D083D0E0BE
:011F59003255
:01246A00323F
:01246B00323E
:01246C00323D
:01246D00323C
:01246E00323B
:01246F00323A
:012470003239
:012471003238
:012472003237
:012473003236
:012474003235
:012475003234
:012476003233
:012477003232
:012478003231
:012479003230
:01247A00322F
:01247B00322E
:01247C00322D
:01247D00322C
:01247E00322B
:01247F00322A
:012480003229
:012481003228
:012482003227
:012483003226
:012484003225
:012485003224
:012486003223
:012487003222
:012488003221
:012489003220
:01248A00321F
:01248B00321E
:01248C00321D
:01248D00321C
:1000E400E4F5C8E58E54074438F58E8FCB8FCDAF39
:0C00F400058FCA8FCCD2BDD2ADD2CA227B
:101F5A00AB07AA06A905A8047F007E1B7D377C4B28
:101F6A0012031CAB07AA06A905A804E4FFFE7D809C
:101F7A007C471202241203B9AD07AC06AF04020073
:011F8A00E472
:1023F500AD07AC06C3E49DFBE49CFFEBFD0200E4E6
:03245700C2CA22D4
:03002B00021AEFC7
:101AEF00C0E0C0F0C083C082C085C084C086758648
:101AFF0000C0D075D000C000C001C002C003C00438
:101B0F00C005C006C00712209EC2CFD007D006D096
:101B1F0005D004D003D002D001D000D0D0D086D0D1
:0C1B2F0084D085D082D083D0F0D0E0328A
:0A00360000010202030304040505A3
:101F8B00EC4EFEED4F2436F58274003EF583E49360
:101F9B00FF3395E0FEEF24A1FFEE34E68F82F5834D
:101FAB002290E6BCE0547EFF7E00E0D394807C0060
:011FBB002203
:03000B00021B3B9A
:101B3B00C0E0C0F0C0D075D000C000C004C005C06C
:101B4B0006C007054BE54BB40621051AE51A7002D2
:101B5B000519AE19FF7C007D0A1204B4ED4C700818
:101B6B000513E51370020512754B00D007D006D094
:0C1B7B0005D004D000D0D0D0F0D0E03273
:10146500E4F529F528F527F526C203C200C202C214
:1014750001121CCF754E01754F0275560175571631
:10148500754C01754D227554017555447558017596
:101495005966D2E843D82090E668E04409F090E622
:1014A5005CE0443DF0D2AFD207121FBC90E680E06D
:1014B50054F7F0C203300105120D1CC20130032997
:1014C5001212FE5024C20312214820001690E68213
:1014D500E030E704E020E1EF90E682E030E604E06A
:0E14E50020E0E412204612245A12227480C71E
:100D1C0090E6B9E07003020DCD147003020E21248D
:100D2C00FE7003020E7B24FB7003020DC7147003CC
:100D3C00020DC114607314607624056003020EB2B8
:100D4C0012245C4003020EBE90E6BBE024FE60223F
:100D5C0014603324FD601114602224067048E54EA3
:100D6C0090E6B3F0E54F8037E55690E6B3F0E557E3
:100D7C00802DE55090E6B3F0E5518023E55290E6E6
:100D8C00B3F0E553801990E6BAE0FF122072AA0680
:100D9C00A9077B01EA494B600DEE90E6B3F0EF90AA
:100DAC00E6B4F0020EBE020EB712242F020EBE12D3
:100DBC002438020EBE120003020EBE122426020EAE
:100DCC00BE12245E4003020EBE90E6B8E0247F60A3
:100DDC00151460192402703AA200E43325E0FFA236
:100DEC0002E4334F8018E490E740F08016121FACF9
:100DFC0040047D0180027D00121F8BE0540190E7BE
:100E0C0040F0E4A3F090E68AF090E68B7402F002D6
:100E1C000EBE020EB71224604003020EBE90E6B85E
:100E2C00E024FE601624026003020EBE90E6BAE0D7
:100E3C00B40105C200020EBE020EB790E6BAE07015
:100E4C002C121FAC40047D0180027D00121F8BE030
:100E5C0054FEF090E6BCE05480131313541FFFE0D3
:100E6C00540F2F90E683F0E04420F08045803C1234
:100E7C002462503E90E6B8E024FE601A24027032E0
:100E8C0090E6BAE0B40104D200802790E6BAE0B450
:100E9C000202801E8015121FAC40047D0180027D71
:100EAC0000121F8B80081211BD500790E6A0E04481
:0A0EBC0001F090E6A0E04480F0226F
:0300330002245054
:0424500053D8EF323C
:1020460090E682E030E004E020E60B90E682E030A5
:10205600E119E030E71590E680E04401F07F147E58
:0C20660000121BD290E680E054FEF02235
:1021480090E682E044C0F090E681F0438701000009
:042158000000002261
:101FBC0030070990E680E0440AF0800790E680E064
:101FCC004408F07FDC7E05121BD290E65D74FFF0B6
:0F1FDC0090E65FF05391EF90E680E054F7F0222B
:08244000E4F55FD2E9D2AF22FE
:101E270090E678E020E6F9C2E990E678E04480F0B1
:101E3700EF25E090E679F090E678E030E0F990E67B
:101E470078E04440F090E678E020E6F990E678E024
:061E570030E1D6D2E922C1
:101EC600A90790E678E020E6F9E55F702390E678CA
:101ED600E04480F0E925E090E679F08D5AAF03A959
:101EE60007755B018A5C895DE4F55E755F01D32247
:021EF600C32205
:101E9200A90790E678E020E6F9E55F702590E678FC
:101EA200E04480F0E925E0440190E679F08D5AAFF4
:101EB20003A907755B018A5C895DE4F55E755F03C2
:041EC200D322C32242
:03004B00020FE2BF
:100FE200C0E0C083C082C085C084C086758600C050
:100FF200D075D000C000C001C002C003C006C00747
:1010020090E678E030E206755F060210CC90E67852
:10101200E020E10CE55F64026006755F070210CC18
:10102200E55F24FE605F14603624FE70030210BD8B
:1010320024FC70030210C9240860030210CCAB5BCD
:10104200AA5CA95DAF5E055E8F82758300120453B0
:1010520090E679F0E55E655A7070755F05806B9079
:10106200E679E0AB5BAA5CA95DAE5E8E8275830019
:10107200120492755F02E55A6401704E90E678E0C0
:101082004420F08045E55A24FEB55E0790E678E0FC
:101092004420F0E55A14B55E0A90E678E04440F048
:1010A200755F0090E679E0AB5BAA5CA95DAE5E8EEF
:1010B20082758300120492055E800F90E678E04408
:1010C20040F0755F008003755F005391DFD007D059
:1010D20006D003D002D001D000D0D0D086D084D0A8
:0810E20085D082D083D0E032FA
:02207200A907BC
:10207400AE58AF598F828E83A3E064037017AD010D
:1020840019ED7001228F828E83E07C002FFDEC3EDF
:09209400FEAF0580DF7E007F0035
:01209D002220
:10229200121E92E55F24FA600E146006240770F3A2
:0C22A200D322E4F55FD322E4F55FD322E1
:1022AE00121EC6E55F24FA600E146006240770F352
:0C22BE00D322E4F55FD322E4F55FD322C5
:101BD2008E2A8F2B90E600E054187012E52B240118
:101BE200FFE4352AC313F52AEF13F52B801590E68F
:101BF20000E05418FFBF100BE52B25E0F52BE52A7A
:101C020033F52AE52B152BAE2A7002152A4E6005F4
:061C120012215C80EE22AD
:10215C007400F58690FDA57C05A3E582458370F996
:01216C002250
:03004300021300A5
:0300530002130095
:101300000220F4000222370002221800022191007C
:10131000021EF800021F290002246A0002246B004A
:1013200002246C0002246D0002246E0002246F006F
:10133000022470000224710002247200022473004F
:101340000224740002246B0002247500022476003B
:1013500002247700022478000224790002247A0013
:1013600002247B0002246B0002246B0002246B0029
:1013700002247C0002247D0002247E0002247F00DF
:1013800002248000022481000224820002248300BF
:10139000022484000224850002248600022487009F
:1013A000022488000224890002248A0002248B007F
:0813B00002248C0002248D00D0
:10022100020425E86480F8E933E83360110460F0E2
:10023100ED33EC337009E8FCE9FDEAFEEBFF220443
:1002410060DED3EB9FEA9EE99DE8C2E78CF0C2F73E
:1002510095F0400CE8CCF8E9CDF9EACEFAEBCFFB0A
:100261001203F085D0F05804700320D5B3E8047070
:10027100075002B2D502042F92D5EC0460F7E4CC0A
:10028100C0E0C398F8603B94186008400DD0E0FBD3
:10029100020407E4FBFAC9FC8028E830E406E4C95B
:1002A100FBE4CAFCE830E305E4C9CACBFCE8540727
:1002B1006010F8C3E913F9EA13FAEB13FBEC13FC32
:1002C100D8F130F52FC3E49CFCEF9BFFEE9AFEEDD5
:1002D10099FDD0E0FBEF4E4D4C701222DB0302047E
:1002E1002CEC2CFCEF33FFEE33FEED33FDED30E76C
:1002F100EB020407EF2BFFEE3AFEED39FDD0E0FBF8
:1003010050130BBB000302042FED13FDEE13FEEFA0
:0803110013FFEC13FC020407CA
:1003190002042FEC5D046005E8590470030204250A
:100329001203F0580460F6EC4860F2EC7004FDFE2C
:10033900FF22C860DB2481C85009C39860025006B7
:1003490002042C9850CAF582E9294B4A7005AB8200
:1003590002041B75F0007C1A7880C3EF9BEE9AEDBE
:1003690099400DC3EF9BFFEE9AFEED99FDE842F02F
:10037900DC23ACF0D0E0FFD0E0FED0E0FDAB822082
:10038900E7101BEB60BAEC2CFCEF33FFEE33FEED0C
:1003990033FD020407E803F830E705C0F075F00003
:1003A900EF2FFFEE33FEED33FD40B830E7C280AAF0
:1003B900EDD2E7CD33EC3392D524814006E4FFFE3C
:1003C900FDFC22FCE4CFCECDCC24E0501174FF809B
:1003D900EDC3CC13CCCD13CDCE13CECF13CF047038
:0703E900F030D5DE0205092A
:1003F000E9D2E7C933E833F892D5EDD2E7CD33EC53
:0704000033FC5002B2D522CB
:10040700EC30E7100FBF000C0EBE00080DBD000456
:100417000BEB6014A2D5EB13FCED92E7FD2274FF02
:10042700FCFDFEFF22E480F8A2D574FF13FC7D805B
:03043700E480EF6F
:030000000214F3F4
:0C14F300787FE4F6D8FD75815F02153AA1
:10043A00BB010689828A83E0225002E722BBFE02C0
:09044A00E32289828A83E49322F3
:10045300BB010CE58229F582E5833AF583E022505E
:1004630006E92582F8E622BBFE06E92582F8E222A8
:0D047300E58229F582E5833AF583E49322C2
:10048000BB010689828A83F0225002F722BBFE015B
:02049000F32255
:10049200F8BB010DE58229F582E5833AF583E8F0A0
:1004A200225006E92582C8F622BBFE05E92582C84C
:0204B200F22234
:1004B400BC000BBE0029EF8DF084FFADF022E4CC2C
:1004C400F875F008EF2FFFEE33FEEC33FCEE9DECF5
:1004D400984005FCEE9DFE0FD5F0E9E4CEFD22ED3B
:1004E400F8F5F0EE8420D21CFEADF075F008EF2F85
:1004F400FFED33FD4007985006D5F0F222C398FD76
:050504000FD5F0EA2212
:0E050900C3E49FFFE49EFEE49DFDE49CFC2203
:0C051700A42582F582E5F03583F58322EF
:10052300D083D082F8E4937012740193700DA3A367
:1005330093F8740193F5828883E47374029368607B
:06054300EFA3A3A380DF7B
:10054900D083D082F8E4937012740193700DA3A341
:1005590093F8740193F5828883E473740293B5F078
:0D056900067403936860E9A3A3A3A380D8E0
:1019B3008B388A39893AE4F540F541E53F153FAE66
:1019C3003E7002153E4E6033AB3BAA3CA93D120468
:1019D3003AFFAB38AA39A93A0541E541AC40700258
:1019E300054014F5828C83EF120492EF60CD7401ED
:1019F300253DF53DE4353CF53C80C0AB38AA39A91B
:021A03003A2285
:1023A900E4FFFE12043A600C0FEF70010E09E970A8
:0523B900F20A80EF2292
:10057600EF4E6012EF60010EEDBB010B89828A839C
:10058600F0A3DFFCDEFA2289F05007F709DFFCA9A9
:0C059600F022BBFEFCF309DFFCA9F02200
:1014FF00021465E493A3F8E493A34003F68001F28A
:10150F0008DFF48029E493A3F85407240CC8C333ED
:10151F00C4540F4420C8834004F456800146F6DFBC
:10152F00E4800B0102040810204080902394E47E95
:10153F00019360BCA3FF543F30E509541FFEE493B1
:10154F00A360010ECF54C025E060A840B8E493A378
:10155F00FAE493A3F8E493A3C8C582C8CAC583CAA3
:10156F00F0A3C8C582C8CAC583CADFE9DEE780BE5B
:0123A8000034
:00000001FF
